:020000040000FA
:1000000002EF00F011EEFFF021EEFFF0F86AA68E8D
:10001000A69C07EEFFF00068ED6A0050FDE11C0EA3
:10002000F66E010EF76E000EF86E0900F5CF05F0C2
:100030000900F5CF06F034D00900F5CF00F0090033
:10004000F5CF01F00900F5CF02F009000900F5CF66
:10005000E9FF0900F5CFEAFF090009000900F5CF23
:1000600003F00900F5CF04F009000900F6CF07F00E
:10007000F7CF08F0F8CF09F000C0F6FF01C0F7FF96
:1000800002C0F8FF03D00900F5CFEEFF0306FBE244
:100090000406F9E207C0F6FF08C0F7FF09C0F8FF41
:1000A0000506CAE20606C8E276EC00F0FFD7E806CD
:1000B000E56E630E6AEC00F0E4500BE000D0E56EF4
:1000C000630E6AEC00F000D000D00000E450E82E8F
:1000D000F6D71200E8060000E85007E000D000D094
:1000E00000D000D00000E82EFAD7120095928C9232
:1000F000006A8CB2002A0050D880E866D890006A66
:1001000000360050010BE844F46E8C50FD0BF410E7
:100110008C6EF40E57EC00F0EBD7120001002A01B0
:0C01200000006000000001000000000072
:020000040030CA
:010001000CF2
:010003001EDE
:010006008178
:00000001FF
